:020000040000FA
:04000000BFEF09F055
:08000800E8CF05F0D8CF06F0A7
:10001000E0CF07F00001E9CF0DF0EACF08F0E1CF23
:1000200009F0E2CF0AF0D9CF0BF0DACF0CF0F3CF22
:1000300014F0F4CF15F0FACF16F000C00FF001C0A5
:1000400010F002C011F003C012F004C013F09DAA1A
:100050002DEF00F09EBA03EF07F0A0AA33EF00F0F7
:10006000A1BAC2EF06F00FC000F010C001F011C03D
:1000700002F012C003F013C004F00DC0E9FF08C085
:10008000EAFF09C0E1FF0AC0E2FF0BC0D9FF0CC0C4
:10009000DAFF14C0F3FF15C0F4FF16C0FAFF05C065
:1000A000E8FF07C0E0FF06C0D8FF1000F76ABC0FEA
:1000B000F66E000EF7220900F5501200040300004E
:1000C0000000000000000000000000000DAE03D0A2
:1000D000F2CF0EF0F29EF76AEE0FF66E000EF722E8
:1000E0000900F5500DAE02D00EBEF28E1200400097
:1000F00040000000000000000000000000000000C0
:100100000000000000000000000000000000F76A8E
:100110001E0FF66E010EF7220900F55012000600C0
:10012000FF0901A101190129081580257F7508958E
:1001300008810219012908750895089102C0F76A1B
:100140004E0FF66E010EF7220900F5501200000066
:10015000F76A600FF66E010EF7220900F5501200E3
:100160002000F76A720FF66E010EF7220900F550B3
:10017000120009022900010100C032090400000236
:100180000300000009210001000122200007058171
:10019000034000010705010340000100F76AAC0FAE
:1001A000F66E010EF7220900F55012000100F76A01
:1001B000BE0FF66E010EF7220900F5501200120173
:1001C0001001000000406104200000010102000154
:1001D000F76AE00FF66E010EF7220900F5501200E3
:1001E0000403090408035300410043001C035300A7
:1001F00065006D00690066006C00750069006400B0
:100200002E0063006F006D00F2CF0EF0F29EF76AD1
:10021000220FF66E020EF7220900F5500EBEF28E86
:1002200012000D0A0A55534220636F6E6E656374A7
:1002300065642C2077616974696E6720666F72202F
:10024000656E756D61726174696F6E00F2CF0EF04C
:10025000F29EF76A660FF66E020EF7220900F5505D
:100260000EBEF28E12000D0A0A55534220646973C5
:10027000636F6E6E65637465642C20776169746961
:100280006E6720666F7220636F6E6E656374696F50
:100290006E00F2CF0EF0F29EF76AAC0FF66E020E11
:1002A000F7220900F5500EBEF28E12000D0A0A5513
:1002B000534220656E756D65726174656420627964
:1002C0002050432F484F53540000F2CF0EF0F29EBF
:1002D000F76AE40FF66E020EF7220900F5500EBE23
:1002E000F28E12000D0A0A55534220756E656E7526
:1002F0006D6572617465642062792050432F484FA8
:1003000053542C2077616974696E6720666F722080
:10031000656E756D65726174696F6E006D9269943A
:100320006894CDEF06F06A6A6892D6EF06F0020193
:10033000596B59530AE1036A5951280FE96E000EAF
:100340000320EA6EEF6A592BF4D71B6A010E1C6E6C
:100350001A6A0001000C010E0201626F62510F085F
:100360000EE3700E6225016E0F0E036ED8B0032AE5
:1003700001C0E9FF03C0EAFFEF6A622BEFD71F6AF3
:100380001E6A0001000C400E0401016F050E036F90
:10039000026B880E006F046B050E076F400E066F30
:1003A0000001000C6A6A686A9F0E6B6E390E696EF6
:1003B0006E6ABDDFD0DF160E706E68A602D068963A
:1003C000FCD76D98E0DF030E206EDCEF06F0698449
:1003D00068986D82E2EF06F0689CE8EF06F070A086
:1003E00002D0D1DF7090689AEEEF06F05DC221F086
:1003F000000CFF0E216E000C02015B6B275234E0F3
:100400005B513F0831E31D50FC0F21E2040F000156
:100410003FEF02F0036A2650A4DEE8CF5CF202014F
:1004200016D0036A265073DEE8CF5CF202010FD0CB
:10043000036A2650CDDEE8CF5CF2020108D0036AE1
:100440002650B5DEE8CF5CF2020101D00201262A77
:1004500027065B515B2B036A400FE96E050E0320F4
:10046000EA6E5CC2EFFFCAD7275204E15B51400835
:1004700001E01A6A5BC25DF20001B8DF000CE824FB
:10048000990FF66E040EF76ED8B0F72A0A00F550F1
:10049000FA6E0800F550F96E1404220430043E048C
:1004A000266A1D6A05010351010A000109E0030AD9
:1004B0000CE0010A0DE0220A1DE0030A28E053D0F7
:1004C000120E276E030E1D6E50D0290E276E4DD0D2
:1004D000020E1D6E036A05010251220FE96E000E25
:1004E0000320EA6EEFCF26F0036A2650000170DE8B
:1004F000276E3BD0120E266E263C01D006D0036A32
:1005000026502FDE276E31D002D073DF3AD0D8903C
:1005100005010435036AF2CF5BF2F29E00010FDEA3
:100520000900F5CF03F002015BBFF28E266E263C78
:1005300001D016D0010E1D6ED89005010435036A56
:10054000F2CF5BF2F29E000103DE0900F5CF03F06B
:1005500002015BBFF28E276E000107D004D00201BA
:10056000000147DF0ED045DF0CD00501075305E140
:100570002750065D02E206C527F0010E1A6E000143
:100580003BDF000C02015A5306E1040E206E00010D
:10059000E2DEC3D00201050E206E5D6F800E5C6F3F
:1005A000010E5B6F5B510F08D8A0B7D05E6B036A7A
:1005B0005B5100017BDD000A57E0040E02015E6F13
:1005C000D8905B35036AF2CF62F2F29E00017EDDC5
:1005D0000900F5CF03F0020162BFF28E5F6F03C026
:1005E00060F25B51080DF350010F016E040E036EB3
:1005F000D8B0032A01C0E9FF03C0EAFF5FC2EFFFE2
:100600005B51080DF350020F016E040E036ED8B05B
:10061000032A01C0E9FF03C0EAFF5DC2ECFFED520F
:100620005CC2EFFFD8905B35036AF2CF62F2F29EB4
:1006300000014CDD0900F5CF03F0020162BFF28E2C
:100640005C2703505D23880E616F60B1618160B3E8
:1006500061835B51080DF3CF01F0040E01C0E9FF87
:10066000EA6E61C2EFFF0001036A02015B51000103
:100670001DDD000A34E002015E835B51080DF3507A
:10068000060F016E040E036ED8B0032A01C0E9FF05
:1006900003C0EAFF5DC2ECFFED525CC2EFFFD890F1
:1006A0005B35036AF2CF62F2F29E00010FDD0900B2
:1006B000F5CF03F0020162BFF28E5C2703505D2389
:1006C0005B51080DF350040F016E040E036ED8B099
:1006D000032A01C0E9FF03C0EAFF400EEF6E0201EA
:1006E0005E51060802E10E0E5E6F036A5B51000167
:1006F000DDDC020802E002015E89700E02015B256A
:10070000016E0F0E036ED8B0032A01C0E9FF03C0CB
:10071000EAFF5EC2EFFF5B2B45D70001E1EF03F07C
:100720000501015100010DE0010A15E0020A20E077
:10073000060A2AE0030A31E00E0A31E0010A37E036
:1007400046D01CC040F50501416B020E02015D6FF1
:1007500000014CDE3ED00501022D07D0010E1C1613
:1007600002015D6B000142DE02D0000142DE31D0A9
:100770000501022D06D01C8202015D6B000136DEF0
:1007800002D0000136DE25D0020E1A6E02C525F019
:1007900002015D6B00012ADE1CD082DE1AD01BC074
:1007A00040F5010E02015D6F000120DE12D005014F
:1007B000025101080AE302C51BF002C55AF200010A
:1007C000E1D602015D6B000111DE000102D011DEF5
:1007D00000D021EF05F01BC05AF2050101510001C4
:1007E00007E00A0A0EE0010A2DE00D0A40E041D0C0
:1007F0000501406B416B020E02015D6F0001F6DDE9
:100800003AD002015A531BE0010E5A5D036A0001FF
:10081000C5DC016E0501045DD8A002D002010FD035
:10082000036A0451280FE96E000E0320EA6EEFCF31
:1008300040F5010E02015D6F0001D8DD02D000011C
:10084000D8DD19D002015A530FE0036A05010451A3
:10085000280FE96E000E0320EA6E02C5EFFF0201C9
:100860005D6B0001C3DD02D00001C3DD04D018DEE2
:1008700002D0BFDD00D021EF05F002015B915ABF2D
:100880005B815A9F5BA10DD0036A5A5100010EDCB7
:10089000000A02E1000E01D0010E016E0DD00CD055
:1008A0000201036A5A51000101DC000A02E1000E54
:1008B00001D0010E016E00D0D4EF04F002015B9173
:1008C0005ABF5B815A9F5BA110D05A51080DF3505B
:1008D000040F016E040E036ED8B0032A01C0E9FFB5
:1008E00003C0EAFF880EEF6E09D05A51080DF3CF0E
:1008F00001F0040E01C0E9FFEA6EEF6A0001E3EFC8
:1009000004F002015B915ABF5B815A9F5BA110D03A
:100910005A51080DF350040F016E040E036ED8B047
:10092000032A01C0E9FF03C0EAFF840EEF6E0AD07C
:100930005A51080DF3CF01F0040E01C0E9FFEA6E31
:10094000840EEF6E0001EBEF04F002015B915ABFE1
:100950005B815A9F5BA110D05A51080DF350040FD0
:10096000016E040E036ED8B0032A01C0E9FF03C074
:10097000EAFFEFCF5CF20AD05A51080DF3CF01F035
:10098000040E01C0E9FFEA6EEFCF5CF25CAF02D06B
:100990005CB502D0000E01D0010E016E0001F7EF30
:1009A00004F004C55AF269D701522EE00501015145
:1009B000010A000105E0020A0BE0030A11E022D05F
:1009C00004C55AF27BD702015D6B00010FDD1CD01C
:1009D00004C55AF296D702015D6B000107DD14D001
:1009E0000501406B416B04C55AF20001AED70152BC
:1009F00003E0010E0501406F020E02015D6F000170
:100A0000F5DC02D0F6DC00D021EF05F00501015144
:100A100000D00001EEDC00D021EF05F01A6A0501DC
:100A200000517F0B000107E0010A06E0030A05E020
:100A3000230A04E004D074D6CED6B3D7E7D7D9DCE6
:100A400000D05BEF06F002015A51080DF3CF01F020
:100A5000040E01C0E9FFEA6EEFCF5CF25B510208C1
:100A600006E15CAD02D05B6B02D0010E5B6F5B51A7
:100A7000030812E1840E5C6F5A51080DF350040F05
:100A8000016E040E036ED8B0032A01C0E9FF03C053
:100A9000EAFF840EEF6E09D05B2D03D0C80E5C6FA9
:100AA00004D05B5302E1880E5C6F036A010E026E94
:100AB0005A51006E05E0D89002360336002EFBD75F
:100AC0000250FF0A006EFF0E031A00501E1603505C
:100AD0001F16D8905A35036AF2CF5FF2F29E0001DA
:100AE00066EC00F00900F5CF03F002015FBFF28E63
:100AF0005D6F03C05EF25A51080DF350010F016E95
:100B0000040E036ED8B0032A01C0E9FF03C0EAFF58
:100B10005DC2EFFF5EB15C815EB35C835A51080D2C
:100B2000F3CF01F0040E01C0E9FFEA6E5CC2EFFFF3
:100B30000001000C02015A51080DF350040F016E20
:100B4000040E036ED8B0032A01C0E9FF03C0EAFF18
:100B5000EFCF5EF25EBF5BD05A51080DF350050F28
:100B6000016E040E036ED8B0032A01C0E9FF03C072
:100B7000EAFF5BC2EFFF5D51020816E15A51080D12
:100B8000F350040F016E040E036ED8B0032A01C0A7
:100B9000E9FF03C0EAFFEFCF5EF25EAD02D05D6B0E
:100BA00002D0010E5D6F13D05D51040810E15A515F
:100BB000080DF3CF01F0040E01C0E9FFEA6EEFCF9C
:100BC0005EF25EAD03D0010E5D6F01D05D6B5D2DF9
:100BD00003D0C80E5E6F04D05D5302E1880E5E6FD5
:100BE0005CB15E815CB35E835A51080DF350040F13
:100BF000016E040E036ED8B0032A01C0E9FF03C0E2
:100C0000EAFF5EC2EFFF010E016E03D000D0000EBE
:100C1000016E0001000C02015A5305E10001C3EC12
:100C200001F010D00201036A010E026E5A51006EEB
:100C300005E0D89002360336002EFBD702501E1274
:100C400003501F120001000C5BC26EFF02015B53D8
:100C500003E0040E206E02D0020E206E000136EF7B
:100C600006F01B6A1A6A25C05BF2EED747EF06F062
:100C700002015A530DE11A2C05D00001FCEC01F0E1
:100C800006D002011A50020803E10001EAD702016E
:100C90000001000C6C300201596F593359331F0E9B
:100CA00059176C5246E1040100513C0B340821E114
:100CB000046B0001B3D6213C07D002015A6B030E2E
:100CC0005B6F0001C0DE12D002015A6B020E5B6F37
:100CD0000001B9DE2150FE0809E002015A6B5C6B8D
:100CE00021C05BF2040E5D6F000124DF6D981ED001
:100CF000040100513C0B04081AE102015A6B000187
:100D00008ADF02015A6B020E5B6F00019CDE2150EC
:100D1000FE080CE0213C01D009D002015A6B5C6B4B
:100D200021C05BF2010E5D6F000104DF040127D0DA
:100D300002016C50040816E1FF0E216E5A6B00018F
:100D400097DF213C01D00AD002015A6B5C6B21C0B5
:100D50005BF2020E5D6F0001EDDE02D0C3EC01F02C
:100D60000DD002016CB406D059C25AF2000153DF13
:100D700005D0020159C25AF200017ADF04010001D4
:100D8000F3EF06F0205201E12FD068522DE068A465
:100D900004D069A402D08EEF01F06DA201D024D05E
:100DA00068A204D069A202D093EF01F068A004D039
:100DB00069A002D0D2EF01F068A804D069A802D0DF
:100DC000E7EF01F068AC04D069AC02D0ECEF01F0C1
:100DD00068AA04D069AA02D0EFEF01F068A604D097
:100DE00069A602D057D76896A19A33EF00F09EAA61
:100DF000FED7ABCF19F0AECF01F019A202D0AB985D
:100E0000AB880000000CF29CF29EF2BEFDD7EFDF33
:100E100001C065F202016551120A000101E02DD006
:100E2000E6DF0150340802E0000E01D0010E02019D
:100E3000676F0001DCDF0150560802E0000E01D0B0
:100E4000010E02016715696F0001D1DF01507808BA
:100E500002E0000E01D0010E020169156B6F000166
:100E6000C6DF0150900802E0000E01D0010E020121
:100E70006B15D8A4FF00000100D0C00EF2129E9A9C
:100E800033EF00F06D6A696A080E6F6E9450300996
:100E90000201946E206A186AF2BE188EF29E00015A
:100EA00097EC01F018BEF28E1F6A1E6A01EF08F07F
:100EB000186AF2BE188EF29E97EC01F018BEF28E00
:100EC0006D6A140E6F6E696A6D86010E206E6CEF8E
:100ED00007F06DB601D0ECD7202C0BD06DBA09D03D
:100EE000686A696AA08AC00EF212110E696E020E5B
:040EF000206E000C64
:1010000041D767DF20500208FCE1FCEF09F0020E37
:10101000EA6E470EE96EEF500EE00F0E016E006AA9
:10102000002EFED7012EFBD78F0E006E002EFED7AE
:101030000000EF2EF2D7000C010E0201476F1BC01B
:1010400048F2475319E0295217E1496B4951000111
:1010500004EC01F00201492B006E00509EA8FED75F
:10106000AD6E290E495DF2E1030E4A6F2E0E9EA869
:10107000FED7AD6E4A2FFAD7475319E1295217E030
:10108000496B4951000126EC01F00201492B006E29
:1010900000509EA8FED7AD6E2B0E495DF2E1030E07
:1010A0004A6F2E0E9EA8FED7AD6E4A2FFAD7485330
:1010B00011E02A520FE1496B4951000149EC01F05E
:1010C0000201492B006E00509EA8FED7AD6E1C0E8B
:1010D000495DF2E1485319E12A5217E0496B495141
:1010E000000165EC01F00201492B006E00509EA842
:1010F000FED7AD6E370E495DF2E1030E4A6F2E0E3C
:101100009EA8FED7AD6E4A2FFAD747C229F048C233
:101110002AF000010BEF0AF002014C51080DF350C8
:10112000020F016E040E036ED8B0032A01C0E9FF5E
:1011300003C0EAFFECCF03F0ED52EFCF51F203C052
:1011400052F24C51080DF350010F016E040E036E64
:10115000D8B0032A01C0E9FF03C0EAFFEF50036AD9
:10116000546F03C055F24C51080DF3CF01F0040E3B
:1011700001C0E9FFEA6EEFCF53F253B1558153B38B
:1011800055835551505D08E303E14F51545D04E22E
:1011900055C250F254C24FF2556B546B5551505DCD
:1011A0001AE303E14F51545D16E251C2E9FF52C206
:1011B000EAFFEFCF58F24EC2EAFF4DC2E9FF58C234
:1011C000EFFF4D2BD8B44E2B512BD8B4522B542BB0
:1011D000D8B4552BE3D74FC201F050C202F0000142
:1011E000FDEF08F047C24CF249C24EF248C24DF240
:1011F0004BC250F24AC24FF28FD702C04BF201C02D
:101200004AF2186AF2BE188EF29E47C25AF2020ED5
:1012100002015B6F000117DC18BEF28E02014AC2A8
:1012200001F04BC202F000011DEF0AF047C249F283
:1012300002014D6B4D5107081BE348C200F04D51B0
:10124000016E04E0D8900032012EFCD70050010B53
:101250004A6F4951010B4B6F4A514B19010B4C6FAF
:10126000D89049334C5302E08C0E491B4D2BE2D7EA
:1012700049C201F00001000C016A026A006A036AB7
:1012800002014E5102E14D5118E0100E4F6FD890FF
:101290004B374C37003603364E51035C02E14D515B
:1012A000005C07E34D51005ED8A003064E51035E7B
:1012B000D880013602364F2FEAD700000001000C1B
:1012C00002014751080DF350040F016E040E036E26
:1012D000D8B0032A01C0E9FF03C0EAFFEFCF4FF205
:1012E0004FBF48D04751080DF350060F016E040E52
:1012F000036ED8B0032A01C0E9FF03C0EAFFECCFB8
:1013000003F0ED52EFCF50F203C051F24E6B4D6B34
:101310004E514B5D1AE303E14A514D5D16E248C25E
:10132000E9FF49C2EAFFEFCF54F251C2EAFF50C2CF
:10133000E9FF54C2EFFF502BD8B4512B482BD8B43F
:10134000492B4D2BD8B44E2BE3D7186AF2BE188E1A
:10135000F29E47C25AF24BC25CF24AC25BF24CC2E6
:101360005DF200019AEC05F018BEF28E015004D037
:1013700000D00201000E016E00017BEF0DF0F86A53
:10138000D09E0D8EEA6AE96AB896190EAF6E260EE7
:10139000AC6E900EAB6EC150C00B0F09C16E070E44
:1013A000B46E196A206A226A040E236E0C0E246E33
:1013B000276A296A2A6AC150C00B0A09C16EC09007
:1013C000C082C084C09EC280880ED56ECD6A000ED9
:1013D000CA6E7F0ECB6EB150480BB509B16EB70E19
:1013E000B1169484BD6ABD6AB1169482BA6ABA6AAB
:1013F0009D8AC00EF21204D62B8002013E6B000EB5
:10140000016EC250C30B0110C26E010E476F000186
:10141000FEDD5FDD11D61B52D8B481EF0DF01EA2A8
:1014200081EF0DF0010E0201476F496B2C0E486FE2
:101430004B6B080E4A6F0001D5D62BA035D00201A8
:101440003C6B3CC247F22CC048F20001EFDE01C009
:101450003CF23CC247F22DC048F2E8DE01C03CF24B
:101460003CC247F22EC048F2E1DE01C03CF23CC271
:1014700047F22FC048F2DADE01C03CF23CC247F22C
:1014800030C048F2D3DE01C03CF23CC247F231C06A
:1014900048F2CCDE01C03CF23CC247F232C048F216
:1014A000C5DE01C03CF202D033C03CF233C03CF296
:1014B00002013C53D8B420D3FF0E346E356E366E25
:1014C000376E386E396E3A6E020E2C5CF10FD8B062
:1014D000C6D20F0F0001B7EF0DF02DC048F22EC09D
:1014E00047F202012D50020814E303E147510008BE
:1014F00010E3346A020E356E2DC036F02EC037F080
:101500003C0E2E24E96E000E2D20EA6EEFCF38F04F
:1015100008D0420E346E020E356E2DC036F02EC04D
:1015200037F09DD22DC048F22EC047F202012D5057
:10153000020816E303E14751000812E33C0E2E2493
:10154000E96E000E2D20EA6E2FC0EFFF346A030E05
:10155000356E2DC036F02EC037F02FC038F00AD0CF
:10156000420E346E030E356E2DC036F02EC037F0AD
:101570002FC038F074D22D3C02D0000E01D0010EE5
:101580000201476F3E512D5C02E1000E01D0010EB9
:10159000471510E02DC03EF23E35006E0036FC0EC1
:1015A0000016C250C30B0010C26E010E476F00013F
:1015B0002EDD0201C282C2B2FED7C4CF3DF2346A30
:1015C000040E356E3DC236F02DC037F048D22DC026
:1015D00048F22EC047F202012D50020850E303E109
:1015E000475100084CE32F3C02D0000E01D0010E01
:1015F000476F3E512F5C02E1000E01D0010E4715EE
:1016000010E02FC03EF23E35006E0036FC0E001694
:10161000C250C30B0010C26E010E476F0001F7DC11
:101620000201B36AB26A406B3F6B2DC003F02EC05B
:1016300001F040512D5C13E303E101503F5D0FE2E7
:101640003C0E3F25E96E000E4021EA6EC282C2B216
:10165000FED7C4CFEFFF3F2BD8B4402BE6D7B25014
:10166000B3CF03F0456F03C046F2346A050E356E02
:101670002DC036F02EC037F02FC038F00AD0420E01
:10168000346E050E356E2DC036F02EC037F02FC0EB
:1016900038F0E5D1346A060E356E020146C236F0E6
:1016A00045C237F0DCD12DC048F22EC047F202010E
:1016B0002D500208D8A073D004E147510008D8A0EB
:1016C0006ED0313C02D0000E01D0010E476F3E516A
:1016D000315C02E1000E01D0010E471510E031C06F
:1016E0003EF23E35006E0036FC0E0016C250C30BB3
:1016F0000010C26E010E476F000189DC02012FC08D
:1017000042F230C041F2406B3F6B2DC003F02EC05F
:1017100001F040512D5C35E303E101503F5D31E2C2
:10172000B36AB26A3C0E3F25E96E000E4021EA6EB4
:10173000C282C2B2FED7C4CFEFFFB250B3CF03F024
:10174000476F03C048F2D8904735496F48354A6F14
:101750004AC24CF249C24BF24E6B030E4D6F000170
:101760008BDD02C04BF201C04AF202014B51425DD7
:1017700004E3E3E141514A5DE0E33F2BD8B4402B61
:10178000C4D7346A0C0E356E2DC036F02EC037F03B
:101790002FC038F030C039F031C03AF00ED0420ED0
:1017A000346E0C0E356E2DC036F02EC037F02FC0C3
:1017B00038F030C039F031C03AF051D12DC048F284
:1017C0002EC047F202012D500208D8A070D004E1CB
:1017D00047510008D8A06BD0313C02D0000E01D098
:1017E000010E476F3E51315C02E1000E01D0010E47
:1017F000471511E031C03EF23E35006E0036FC0E5A
:101800000016C250C30B0010C26E010E476F0001DC
:1018100007EC08F002012FC044F230C043F2406BE5
:101820003F6B2DC003F02EC001F040512D5C31E321
:1018300003E101503F5D2DE2B36AB26A3C0E3F25E1
:10184000E96E000E4021EA6EC282C2B2FED7C4CF5A
:10185000EFFFB250B3CF03F0476F03C048F248C266
:101860004CF247C24BF2050E4E6FDC0E4D6F00017D
:1018700003DD02C049F201C048F202014951445D52
:1018800004E3E7E14351485DE4E33F2BD8B4402B48
:10189000C8D7346A070E356E2DC036F02EC037F02B
:1018A0002FC038F030C039F031C03AF00ED0420EBF
:1018B000346E070E356E2DC036F02EC037F02FC0B7
:1018C00038F030C039F031C03AF0C9D00201406B75
:1018D0003F6B405101080BE33C0E3F25E96E000EC3
:1018E0004021EA6EEF6A3F2BD8B4402BF2D7346A1E
:1018F000080E356EB4D00201406B3F6B40510108B9
:101900000CE33C0E3F25E96E000E4021EA6E2DC02F
:10191000EFFF3F2BD8B4402BF1D7346A090E356E58
:101920002DC036F09CD02B80346A0A0E356E020131
:1019300096D02B90346A0B0E356E020190D0346A2B
:101940000D0E356EFF0E936E81CF36F0020187D0FB
:10195000936A2DC08AFF346A0E0E356E2DC036F0A4
:1019600002017DD0346A0F0E356E2DC036F02D5039
:10197000F80F2BE2080F83EF0DF09380376A81B0E8
:10198000372A23D09382376A81B2372A1ED09384B4
:10199000376A81B4372A19D09386376A81B6372AD5
:1019A00014D09388376A81B8372A0FD0938A376A60
:1019B00081BA372A0AD0938C376A81BC372A05D07E
:1019C000938E376A81BE372A00D0020148D02D504D
:1019D000F80F3BE2080F9DEF0DF02EB002D08A9079
:1019E00001D08A80939031D02EB002D08A9201D05B
:1019F0008A8293922AD02EB002D08A9401D08A840F
:101A0000939423D02EB002D08A9601D08A869396E2
:101A10001CD02EB002D08A9801D08A88939815D015
:101A20002EB002D08A9A01D08A8A939A0ED02EB014
:101A300002D08A9C01D08A8C939C07D02EB002D011
:101A40008A9E01D08A8E939E00D0346A100E356E25
:101A50002DC036F02EC037F0020101D002012BA0BC
:101A60003DD03C6B3CC247F234C048F2000116EC5A
:101A700009F001C03CF23CC247F235C048F216EC16
:101A800009F001C03CF23CC247F236C048F216EC05
:101A900009F001C03CF23CC247F237C048F216ECF4
:101AA00009F001C03CF23CC247F238C048F216ECE3
:101AB00009F001C03CF23CC247F239C048F216ECD2
:101AC00009F001C03CF23CC247F23AC048F216ECC1
:101AD00009F001C03CF23CC23BF00201010E476F2D
:101AE000496B340E486F4B6B080E4A6F020E4C6FF9
:101AF000000160EF09F00201010E476F000107ECE1
:101B000008F087D40300F2CF0EF0F29EE8242B0FEA
:101B1000F66E1B0EF76ED8B0F72A0A00F550FA6E73
:101B20000800F5500EBEF28EF96E7A1984198E19DE
:101B30009819A219AC19B619C019F2CF0EF0F29E7D
:101B4000E8245F0FF66E1B0EF76ED8B0F72A0A0076
:101B5000F550FA6E0800F5500EBEF28EF96EDA19E5
:101B6000E819F619041A121A201A2E1A3C1AF2CF82
:101B70000EF0F29EE824930FF66E1B0EF76ED8B0AF
:101B8000F72A0A00F550FA6E0800F5500EBEF28EE4
:101B9000F96EDA1424157615CE159416BC17CC18E8
:101BA000F61826193219A6163E1950196419CE19BD
:020000040030CA
:0E000000240E3F1E008381000FC00FE00F4052
:00000001FF
